:020000040000FA
:04000000FA3060284A
:080008008612601C8616BA0086
:10001000030EBB008312051E21285008E000510882
:10002000E1005208E2005308E3005408E4005508D8
:10003000E5005608E6005708E700601C86166018C1
:100040008612051D2528BC0B21282830BC000F3046
:10005000A9008B100314851E031040193428C01802
:100060003828401839283A28E70CE60CE50CE40C4F
:10007000E30CE20CE10CE00C3B0E8300BA0E3A0EEE
:02008000090075
:1000C000203084008001840A80300402031C6228EE
:1000D0002830BC008316FF3085051F308605C730E9
:1000E00087058312850186018701103083168E00F3
:1000F0008312703083168F0083120030031799002B
:100100000313003003179A000313003097000030E8
:100110009F00003083169F008312003003179E005B
:100120000313003003179F000313C73083168100A9
:10013000831230309000003092000030831694001B
:10014000831200309400A63083169800831200308A
:1001500083169B0083120030980033308316990079
:100160008312003083168C008312003083168D00BA
:10017000831210308B00C20BBB280130AA00810112
:100180008E018F010B118B100B108C128C018D01C5
:100190008B1764000B19CE20DE20C9280B11AA0B87
:1001A00008000430AA000421A9080319DA2806135C
:1001B000A9030800060940398600080003108718C3
:1001C0000314C80D48120C304802031D0800C80172
:1001D000061EF9284F08031DF72841180C21C118E5
:1001E000132141191C21C11933214A08CE002030A6
:1001F000CF00CF03031007190314CD0CCC0CCB0C8C
:10020000CA0C0800431408000130871F0430C100E5
:100210000310071FC10D08000030C0004A08D000BD
:100220004B0AD10008000130C0004A08D0004B0A38
:10023000D1004D08D20008000230C0004A08D000AA
:100240004B0AC200D801D901DA010314D80DD90D27
:10025000DA0D0310C20B26295808D1005908D20024
:100260005A08D3000800CE1F3829CA1F08003A29AF
:10027000CA1B08000430C0004A08D0004B0AC20064
:10028000D801D901DA010314D80DD90DDA0D031004
:10029000C20B44294D08D700CA1F5829D101D201E9
:1002A000D3015808D4005908D5005A08D6000800D0
:1002B000D401D501D6015808D1005908D2005A08F6
:1002C000D30008000708203A870008000708103A02
:0C02D000870008000708083A87000800B3
:084000000800000000000600AA
:02400E00CC03E1
:00000001FF
